:10000000830100308A004428F30003088301DD00E7
:100010000408DE000A08DF008A017008E4007108A5
:10002000E6007208E5006008E2006108E3000B1DCD
:100030001E2808308312031381070B110B1C2B2879
:100040000130C2230030652599247008C50071086D
:10005000C60052270B108B1C30280130C2238B1096
:1000600035236408F0006608F1006508F2006208B4
:10007000E0006308E1005E0884005F088A005D0814
:100080008300F30E730E0900203084005D3052208F
:10009000203084004030831752208301E42D040671
:1000A0008001840A0406031D4F28003483120313C1
:1000B000E000E11B6428611B6C2861088A0060086D
:1000C000E00A0319E10A82008313611883176008AC
:1000D000E00A840000080800533451344F344E3491
:1000E000003455344E344B344E340034533443349E
:1000F00041344E340034533451344F344634003498
:10010000423441344E344B343A34003446343A3479
:10011000003444344134543441343A3400344234A9
:100120002E34563445344C344C3445342034283441
:1001300043342934323430343134313400344C34A3
:1001400042342D343734343430342034563430345F
:080150002E3435343034003444
:10066A006300830108000D3066230A30662B83017C
:10067A00A5003A30662325084C233D30662B8312A9
:10068A00C80083169B001C141A08831208008301F1
:10069A00CC004C0E0F396F234C080F396F2B830196
:1006AA00D5000730D6005408D7005508852E080013
:1006BA008301BD000730BE003C08BF003D08342E50
:1006CA0008008301CF00831203130C1E682B4F0806
:1006DA00990008008301CD000A304D020318772BD8
:1006EA003030782B3730CD074D08662B8301A500B3
:1006FA00822BA50A25034423662383120313A50329
:10070A00250F7E2B08008301CE017D30C223992458
:10071A00F11F0134CE0A18304E02031800348A2B16
:10072A008301D4008730D7004030D8005408102401
:10073A00F000F1017104031D01340034AC2B4D08A3
:10074A00E1004C08CC0A0319CD0A5620662383120D
:10075A000313CE034E0FA42B0800831603130516AA
:10076A0000000000000000000000851500000000E5
:10077A00000000000000831208008301CF004F0828
:10078A00A3006E30A400000000000000000000007A
:10079A000000A40BC82BA30BC62B08000000000006
:1007AA000000831603130516000000000000000075
:1007BA00000083120512831605120000000083123E
:1007CA0008008301D500540BED2B1030D600EE2B18
:1007DA00D6018930D7005608D80055081024F000F1
:1007EA00F1017104031D013400348301851183165C
:0607FA00851583120512B3
:1008000083160516831285118316851100000000DA
:1008100083120512831605120000000083120800DF
:100820008301D900FA235908CA24003803191A2C65
:10083000B22301345708CA2400380319212CB223EB
:1008400002345808CA2400380319282CB223033470
:10085000B22300348301A500A701442C250884009D
:100860008313270827070007A600FA232608CA24AF
:100870000038031D422CB223250884008313260868
:1008800080000134B223A70A250827020318003488
:100890002E2C073083019F0083168113D8308500EA
:1008A000FD30860024309800903083129800193073
:1008B0008316990083129A019A019A018B13831669
:1008C0008112FA30831281000B168B1505148514E2
:1008D000051508008301A50000308B1B0130A60020
:1008E0008B13FA232508CA24003803197A2CB22363
:1008F0000130972C2508CA2400380319822CB22312
:100900000230972CFA23250ACA24003803198B2CAD
:10091000B2230330972C2608840083130030FC2474
:1009200083138000B2238B1326188B1700308301AA
:10093000080083010608F039CF00B92CFF30F00021
:10094000F1000800F001F10108000130F000003072
:10095000F10108000230F0000030F101080003301E
:10096000F0000030F1010800FE30F000FF30F1002F
:1009700008004F08703A0319A22CC03A0319A52C9D
:10098000603A0319AA2C303A0319AF2C103A031914
:100990009E2CB42C8301DB00DC01DB1FD22C8316E0
:1009A0008515D52C851183168511D3230310DB0DF6
:1009B000DC0A08305C02031CCD2C83168515000070
:1009C0000000000005160000000000000030831247
:1009D00085190130DA0000000000051283160512A7
:1009E00000000000000083128511831685110000AD
:1009F000000083125A0808008301C200C401831654
:100A0000851508308312C3000310C40D8316051624
:100A100000000000000083128519C40A00000000D5
:100A200005128316051200000000000000000000FF
:100A30008312C30B042DC2080319222D85118316BE
:100A40008511242D8316851500000000D323851100
:100A5000831685110000000000008312440808007E
:100A60008301A50026087F39F0000310F00C031065
:100A7000700CF0002508F1000530F2000310F10DB4
:100A8000F20B3E2D71087004A70027083F39F000D3
:100A90002608F1000630F2000310F10DF20B4C2D88
:100AA00071087004A8002808A9002908AA002A08CB
:100AB000AB002B08AC002730D40025085423A60037
:100AC000A60803190034260808008301C50005089C
:100AD000F0000630F1000310F00CF10B6B2D7008E4
:100AE000C600450B742D782D4608210603199C2D50
:100AF0004608A100C7012108F0000530F1000310ED
:100B0000F00DF10B7F2D700847074423F0004708D4
:100B1000203E8400831770088000C70A20304702F7
:100B2000031C7B2D8030CC000030CD000530CE0082
:100B3000A32321084C233823210808008301B40093
:100B40003630BC0034085D23B500B5080319AA2D62
:100B5000350808002D08840083133608F00005309E
:100B6000F1000310F00CF10BB12D700880002E087D
:100B7000840083133708F0000630F1000310F00CF6
:100B8000F10BBE2D7008F00036081F39F10003107C
:100B9000F10D0310710D700480002F088400831381
:100BA00037083F3980003008840038088000310859
:100BB000840039088000320884003A088000330835
:100BC00084003B0880000034492438239F30CC0047
:100BD0000030CD000C30CE00A32338238F30CC0062
:100BE0000030CD000F30CE00A3233823AA30A00060
:100BF0002630AD002730AE002C30AF002B30B000D7
:100C00002A30B1002930B2002830B30020089E25D8
:100C1000A5008930CC000030CD000530CE00A323E4
:100C200025084C233A30662326084C233A306623A5
:100C300027084C233A3066232C084C232B084C23DE
:100C40002A084C2329084C2328084C23382338230E
:100C50000130652599247008C5007108C600522727
:100C60008B1763008301332E8301C00000308B1B80
:100C70000130C1008B13FA234008CA24003803193D
:100C8000442EB2230130832E3E08CA2400380319B3
:100C90004C2EB2230230832EFA23400ACA24003895
:100CA0000319552EB2230330832E3F08840083138B
:100CB0000130FC24831380003F0A84000130FC24AF
:100CC000831380003F08023E84000130FC2483131C
:100CD00080003F08033E84000130FC248313800021
:100CE0003F08043E84000130FC24831380003F0849
:100CF000053E84000030FC2483138000B2238B1354
:100D000041188B170030830108008301D8000030A0
:100D10008B1B0130D9008B13FA235808CA240038E2
:100D20000319952EB2230130E82E5608CA24003844
:100D300003199D2EB2230230E82E57088400831336
:100D40000008CA2400380319A82EB2230330E82E65
:100D5000570A840083130008CA2400380319B32EED
:100D6000B2230430E82E5708023E840083130008A3
:100D7000CA2400380319BF2EB2230530E82E5708C5
:100D8000033E840083130008CA2400380319CB2EC5
:100D9000B2230630E82E5708043E8400831300086F
:100DA000CA2400380319D72EB2230730E82E57087B
:100DB000053E840083130008CA2400380319E32E7B
:100DC000B2230830E82EB2238B1359188B1700304A
:100DD000830108008301CC00F72E05148510F22E44
:100DE000051085140511092F05108510082F831291
:100DF00003134C08203E8400831700080319ED2ECE
:100E0000013A0319F02E033A0319F42E0514851440
:100E100005154C0A203E840083170008CE004C08BC
:100E2000023E203E84000008CF004C08033E203ED6
:100E300084000008D0004C08043E203E84000008D6
:100E4000D1004C08053E203E84000008D2004C082A
:100E5000063E203E84000008D300D401D40A2008B6
:100E6000E623CD00CD080319372F4D0808004E307A
:100E7000D40020085423CD00CD080319412F4D087C
:100E80000800D4012008E623CD00CD0803194A2F1D
:100E90004D08080020089523CD00CD080319003423
:100EA0004D0808008301460AFE3003194506031D5C
:100EB000652F7130CC000030CD000530CE00A3236B
:100EC0003823FF30C500C6000800450A0319460A4A
:100ED000031DED2F7630CC000030CD000530CE0064
:100EE000A32338238630CC000030CD000230CE0062
:100EF000A323CA014A08F0000310F00D0310F00DFF
:100F00000310700DC800073E203E84008317000BBD
:100F10008A2FDE2F4808EA268317C7004A084C2389
:100F20002F30662347084C232D3066230A30C22316
:100F3000003086190130CB002830C22300308619DA
:100F40000130CB073230C223003086190130CB0785
:100F50001930C223003086190130CB071930C22363
:100F6000003086190130CB0704304B02031CD22F0E
:100F7000C908031DC62F6C30CC000030CD000430F2
:100F8000CE00A3233A306623C901C90A4508CC0024
:100F90004608CD008823F000F10171040319861D75
:100FA000D22FB82F490BDE2F7B30CC000030CD0084
:100FB0000430CE00A3232D306623C9019924700884
:100FC000C5007108C600C61BE72F3823ED2F04307B
:100FD000CA0A4A02031C7A2F792F8630CC000030CF
:100FE000CD000230CE00A32345084C23382345080A
:100FF000F0000310F00D0310F00D0310700DEA2E39
:02400E00383F39
:1042000001004100C200CA00E20094005300000017
:104210000000A10043000B004800D500440000004E
:104220000000A1004200DF00CA00930091000000DE
:104230000000A1004200ED006800150036000000FB
:104240000000A10043000B004800D500440000001E
:104250000000A1004200E400540069007300000067
:104260000000A1004200F7009E003600720000002E
:104270000000A10043000300B8007000CC00000063
:104280000000A10043000B004800D50044000000DE
:104290000000A1004200FB0005009600DC000000C9
:1042A0000000A1004200F700C400F000C7000000B9
:1042B0000000A10043000300B8007000CC00000023
:1042C00001004100C200E400440046007B00000001
:1042D0000200E000C200C600C700EE003E00000081
:1042E0000000A1004200F400F8007900AF000000D7
:1042F0000000A10043000300B8007000CC000000E3
:00000001FF
